:0200000480007A
:100000006F008004732F2034930F80006308FF0378
:10001000930F90006304FF03930FB0006300FF038E
:10002000130F000063040F0067000F00732F2034CC
:1000300063540F006F00400093E19153171F0000BD
:1000400023223FFC6FF09FFF93000000130100008C
:10005000930100001302000093020000130300004C
:100060009303000013040000930400001305000034
:10007000930500001306000093060000130700001C
:100080009307000013080000930800001309000004
:1000900093090000130A0000930A0000130B0000EC
:1000A000930B0000130C0000930C0000130D0000D4
:1000B000930D0000130E0000930E0000130F0000BC
:1000C000930F0000732540F16310050097020000B4
:1000D000938202017390523073500018970200000F
:1000E00093824202739052309B021000939252030B
:1000F0009382F2FF7390023B9302F0017390023AF5
:100100007350403097020000938242017390523046
:10011000735020307350303093010000970200007C
:10012000938282EE73905230130510001315F5017F
:10013000635C05000F00F00F930110009308D005D9
:10014000130500007300000093020000638A0200A0
:1001500073905210B7B200009B82921073902230BD
:100160007350003097020000938242017390123462
:10017000732540F17300203097200000938080E8C1
:1001800003D700009303F00F930120006316772636
:1001900097200000938000E703D72000B7030100F9
:1001A0009B8303F0930130006318772497200000AD
:1001B000938040E503D74000B71300009B8303FF03
:1001C00093014000631A772297200000938080E318
:1001D00003D76000B7F300009B83F3009301500046
:1001E000631C772097200000938020E203D7A0FFB4
:1001F0009303F00F930160006310772097200000B5
:100200009380A0E003D7C0FFB70301009B8303F0F6
:10021000930170006312771E972000009380E0DE48
:1002200003D7E0FFB71300009B8303FF9301800017
:100230006314771C97200000938020DD03D7000013
:10024000B7F300009B83F300930190006316771AC5
:1002500097200000938000DB938000FE83D2000291
:100260009303F00F9301A000639872189720000089
:10027000938040D99380B0FF83D27000B703010010
:100280009B8303F09301B000639872169301C00042
:1002900013020000972000009380E0D603D72000CF
:1002A00013030700B71300009B8303FF6316731447
:1002B0001302120093022000E31E52FC9301D000AF
:1002C0001302000097200000938000D403D7200081
:1002D0001300000013030700B7F300009B83F30033
:1002E000631C73101302120093022000E31C52FCE3
:1002F0009301E0001302000097200000938080D05B
:1003000003D72000130000001300000013030700B0
:10031000B70301009B8303F06310730E13021200F6
:1003200093022000E31A52FC9301F0001302000034
:1003300097200000938020CD03D72000B713000042
:100340009B8303FF631A770A1302120093022000B3
:10035000E31052FE930100011302000097200000F9
:10036000938080CA1300000003D72000B7F3000079
:100370009B83F3006312770813021200930220009C
:10038000E31E52FC930110011302000097200000AD
:10039000938040C7130000001300000003D7200023
:1003A000B70301009B8303F0631877041302120064
:1003B00093022000E31C52FC97220000938282C427
:1003C00003D10200130120009303200093012001B8
:1003D00063147102972200009382C2C203D102000B
:1003E000130000001301200093032000930130014B
:1003F00063147100631030020F00F00F638001007E
:100400009391110093E111009308D0051385010029
:10041000730000000F00F00F930110009308D00547
:100420001305000073000000731000C000000000FE
:0C043000000000000000000000000000C0
:1010000000000000000000000000000000000000E0
:1010100000000000000000000000000000000000D0
:1010200000000000000000000000000000000000C0
:1010300000000000000000000000000000000000B0
:081040000000000000000000A8
:10200000FF0000FFF00F0FF00000000000000000D4
:040000058000000077
:00000001FF
